:1000000080190020090A00004B470000F509000094
:10001000F5090000F5090000F509000000000000E6
:10002000000000000000000000000000BD0B000008
:10003000F509000000000000890B0000F509000030
:10004000490D0000490D0000490D0000490D000058
:10005000490D0000490D0000490D0000490D000048
:10006000490D0000490D0000490D0000490D000038
:10007000490D0000490D0000490D0000490D000028
:10008000490D0000490D0000490D0000490D000018
:10009000490D0000490D0000490D0000490D000008
:1000A000490D0000490D0000490D0000490D0000F8
:1000B000490D0000490D0000490D0000490D0000E8
:1000C000490D0000490D0000490D0000490D0000D8
:1000D000490D0000490D0000490D0000490D0000C8
:1000E000490D0000490D0000490D0000490D0000B8
:1000F000490D0000490D0000490D0000490D0000A8
:10010000034613F8012B002AFBD1181A0138704757
:100110002DE9F3411C4DAC68E36B13BBE36A3BBBB9
:10012000DFF86480194C1A4EAB681B69EBB10122F1
:100130000DF1070140469847012816D19DF8072088
:100140000A2A01D00D2A18D12368002B15DD0027BB
:10015000F7540F490F480022002302F04BFE27609E
:10016000E2E7284698470028D8D102B0BDE8F081E0
:10017000054898470028D3D1F7E723681E2B9EBF78
:10018000591CF2542160CFE7185200007803002078
:10019000500B002090010020F8B50646FFF7B0FF95
:1001A000064F05460024AC4200DBF8BD315DBB685C
:1001B00002485B6898470134F5E700BF1852000019
:1001C00070B588B01B4C204604F0CCFD28B91A4805
:1001D00004F0CBF9002008B070BDA56825B32B6CE6
:1001E00013B316490022204698472B6AF3B91448E6
:1001F000144C154D154EFFF7CFFF1548FFF7CCFFF8
:100200004FF0FF324FF0FF336946204602F042FEC6
:100210000028DFD12846FFF7BFFF6846FFF7BCFF85
:100220003046FFF7B9FFEBE70A48D1E72046984789
:10023000DDE700BF18520000C455000011010000A6
:100240000E560000900100204F5600002756000077
:100250002A560000DB550000014B1B68184700BF01
:100260000000002030B585B004460D461022002164
:10027000684604F00DFF02238DF802302A46044B35
:1002800001932146684603F031FE05B030BD00BF42
:100290005902000080B505460E461746984603F001
:1002A0003DFA034604F060FFDFF81890044649F871
:1002B0000030424630463946A84754F8090000F05D
:1002C00011FC00BF080000002DE9F047058B044633
:1002D0002807904611D4022905F0070540F0CC808C
:1002E000204604F04FF978B10138218B042811D849
:1002F000DFE800F0C2106D85950001290CBF45F0C4
:10030000100545F02005258388F31188BFF36F8F12
:10031000BDE8F08701F0070AAA4500F0A580002794
:10032000B9463E46A368002B00F0BC8041F00801AE
:10033000218388F31188BFF36F8FA168002900F033
:10034000BA800D68002900F0B680D1F804803346E9
:1003500052462046C047002D76D02B6829461D46C0
:10036000F0E701F007035A1F012A1BD8002221F0F1
:100370000701062B276889B2C4E9002209D13B4650
:1003800003E0628B013262831B68002BF9D141F0DC
:1003900002012183204604F0F5F800287AD041F0CC
:1003A000200176E0042B0AD121F0070189B22183D4
:1003B000204604F0E7F810B141F020012183218BA1
:1003C00001F0070AAA454FD00027B946AAE72369DA
:1003D00021F0070141F00601062DD3F8009021839A
:1003E0002DD1B9F1000F3FD041F00801218388F3EE
:1003F0001188BFF36F8F3A492046C84729E021F0A2
:100400000701236941F0040189B2042DD3F8049057
:100410002183E6D000273E464FF0040A82E721F010
:100420000701236941F0050189B2052DD3F8089031
:100430002183D6D000273E464FF0050A72E70027F9
:100440003E464FF0060A6DE72B4687E7B9F1000FED
:10045000D1D1EFF31188202383F31288BFF36F8F7C
:10046000238B23F008032383258BEA062ED525F062
:100470001003238305F007056669218B002EBFF664
:1004800070AF00232768C4E9003321F0070141F071
:1004900001012183218B01F0070AAA454FF00009D1
:1004A0007FF440AF002F9CD041F00801218388F3F6
:1004B0001188BFF36F8F002FC8D03D68394633468F
:1004C0005246204604F08AF82F46F4E7AB067FF543
:1004D0001BAF25F02003238305F0070500E700BFCD
:1004E00009460000014B036000207047B85300002C
:1004F00008B5044804F039F8BDE80840024804F0A3
:1005000034B800BF565600008B560000014803F077
:1005100045BB00BFB853000038B5044618B90F4BAF
:100520000F485B6898476168B1F5683F10D0B1F536
:10053000680F0DD00B4DA9420AD011F468612068F4
:1005400007D00146084804F068FC0023236065607A
:1005500038BD142204F09CFDF9E700BFD80000204C
:10056000B95600002C5F5CA97C08002008B520B3B8
:100570004368B3F5683F10D101220368BFF35B8F76
:1005800053E8001F002903D143E800200028F7D1D9
:10059000BFF35B8F0DD1002008BD094A93420AD0FA
:1005A00000684FF0FF324FF0FF3302F0CBFC002821
:1005B000F1D00448F0E70448EEE76FF4E040EBE7E1
:1005C0002C5F5CA9E98FFFFFEA8FFFFF08B5D8B168
:1005D0004368B3F5683F10D100220368BFF35B8F17
:1005E00053E8001F012903D143E800200028F7D178
:1005F000BFF35B8F0BD1002008BD074A934208D0A0
:10060000006802F017FDF6E76FF4E040F4E70348F6
:10061000F2E70348F0E700BF2C5F5CA9E98FFFFF1A
:10062000EA8FFFFF10B5044618B91D4B1D485B68E3
:1006300098476368B3F5683F2FD0B3F5680F2CD0A7
:10064000194A934219D1236803BB18484FF0FF326F
:100650004FF0FF33214602F09FFB08B923681BB916
:100660000F4B13485B68984720681422002104F060
:100670000FFD4FF46863636008E0B3F5683F0DD881
:100680003A2B03D040F6BA629342DED1206804F0E0
:10069000FCFB636843F03A03636010BD054AF3E76F
:1006A000D8000020B95600002C5F5CA97C0800200F
:1006B000DF5600003A00003A08B5064906484023D4
:1006C000142204F09CFBBDE808400449044803F0F0
:1006D000D7BA00BF7C0300207C080020C053000074
:1006E000D453000030BFFFF7FDBF00BF2DE9F0413C
:1006F0000B4EDFF8308006EB0807CC1B0546324670
:100700000949204604F0B6FCA01942460021083CE5
:1007100004F0BEFC2C6707F10800BDE8F08100BFC3
:100720000000000004000000AC530000074A93687A
:1007300093F90E10002907DB526993421FBF044A48
:10074000536843F080535360704700BF480900204E
:1007500000ED00E070B5264B15469A6A12F0100FB6
:100760009A6A14BF1124102412F0080F9A6A18BF55
:100770001224920706460AD5586B9A6A140634D595
:1007800019B19A6A22F080029A62132401E06FF094
:100790001500174B9A6A12F0010F9A6A18BF1424B9
:1007A00012F0200F9A6A18BF1524D20602D49B6A51
:1007B0009B070AD50E4B5B68190506D5314600F03C
:1007C00079FA10B180F309880224094B9A6A9206DB
:1007D00042BF5A6A22F400525A629A6A42F0FF02F9
:1007E0009A6200232B70204670BD6FF01500CCE795
:1007F00000ED00E0134B9A6A12F0007F9A6A14BF72
:100800001E201D2012F0807F9A6A18BF1F2012F44C
:10081000002F9A6A18BF212012F4802F9A6A18BFFD
:10082000222012F4003F9A6A18BF232012F4803F5E
:100830009A6A6FEA02426FEA12429A6218BF242053
:10084000704700BF00ED00E010B5194B0246986AF2
:100850009C6A10F4805F14BF1720162014F4006FF8
:100860009C6A18BF1820A40509D5986B986A0004E3
:1008700004D51AB19A6A22F400429A6219200C4BEC
:100880009A6A12F4806F9A6A18BF1A20D2050CD4A3
:100890009B6A13F4005F18BF1C20054A936A43F457
:1008A0007F43936200230B7010BD1B20F5E700BF50
:1008B00000ED00E0F0B5484B5B688BB00446C3F335
:1008C0000803002585F31188BFF36F8F02F07F4086
:1008D000B0F17F4F11D102F00C0008280DD01007A5
:1008E0004CBF0C4601250022033B8DF80720032B4B
:1008F00005D8DFE803F0246367602C46F3E70023A4
:100900009DF80720CAB902AE04F12007206861688B
:10091000324603C20834BC421646F7D1099A002D6C
:1009200054D0C2F3080121B96FEA52226FEA422281
:10093000099202A9184603F0FEFE0BB0F0BD264B4B
:10094000DA6A9107DBD4DA6A002AD8DBDA6A520065
:10095000D5D55A69A16942F480725A61BFF34F8FAD
:10096000BFF36F8F5A6931F8021C22F480725A610A
:10097000BFF34F8FBFF36F8F4DF6027291420AD0D3
:100980009A6AD2B24AB10DF1070201212046FFF75F
:10099000E1FE0346B4E72368B2E79A6A12F47F4F98
:1009A00005D00DF107010120FFF74EFFF1E79B6A2B
:1009B000B3F5803FA3D3FFF71DFFEAE70DF1070270
:1009C0000021E3E70DF107010020EDE722F4FF72BB
:1009D00022F00102ACE700BF00ED00E0044B5A69D1
:1009E00042F010025A615A6922F008025A617047B7
:1009F00000ED00E0EFF30880EFF3098101B57246E6
:100A0000FFF758FF01BD00BF002080F31488BFF33B
:100A10006F8F01F03DFA00200D490860BFF34F8F42
:100A20000C4880F3088800F02BF8202080F3118810
:100A300009484FF40461401880F30988EFF31480EB
:100A40000221084380F31488BFF36F8F00F0FAF897
:100A500094ED00E080190020C00B00200749D1F878
:100A600090200023C2F307221846934200DB704710
:100A7000C1F89830C1F8A0000133F6E700ED00E0BE
:100A800008B572B6002383F31388FFF7E7FF144B12
:100A90004FF0FF32C3F88020C3F88420C3F88820C9
:100AA000C3F88C20C3F89020C3F89420C3F8982092
:100AB000C3F89C20C3F88021C3F88421C3F888219F
:100AC000C3F88C21C3F89021C3F89421C3F898216E
:100AD000C3F89C2162B6BFF34F8FBFF36F8F08BD81
:100AE00000E100E0084B9B6883420BD1EFF30583E4
:100AF00043B1064B5A6842F080525A605A6A22F457
:100B000000425A6204F073BA4809002000ED00E088
:100B1000094A93686FF00A019967084958674B685A
:100B200043F080534B60002383F31188BFF36F8F32
:100B30009368986F704700BF4809002000ED00E0FF
:100B400010B50446EFF31183202383F31288BFF31B
:100B50006F8F0A4B58699860094B4FF000625A60DA
:100B6000084B026F1A600022436F426783F31188BB
:100B7000BFF36F8F00F006F9204610BD4809002032
:100B800000ED00E0980800200B498A684FF0300023
:100B90001044EFF3098C80E8F01F74467046FFF7AD
:100BA000CFFFA64604498A6802F1300090E8F01FA2
:100BB0008CF3098870470000480900201EF0040FDC
:100BC0000CBFEFF30880EFF30980816911F8021C74
:100BD0000229FFD001B503F0B4FD01BD40B20028E9
:100BE00007DB044A4109012300F01F00834042F85B
:100BF0002130704700E100E0054B420900F01F0082
:100C000053F82220012303FA00F01040704700BF80
:100C100000E100E040B20028A8BF00F1604001F10F
:100C20000101B8BF064B4FEA4111ACBF00F561406E
:100C300000F00F00C9B2B4BF195480F80013704718
:100C400014ED00E00B4A08B50B4B22F07F029A60CE
:100C5000BFF34F8FBFF36F8FD3F8882022F4700259
:100C6000C3F8882001F0D4FF02F0E4FD00F060F842
:100C700002F012F80000000000ED00E042F8203C15
:100C8000009B42F81C3C0A49019B42F8183C029B1D
:100C900042F8143C21F001014FF0807342F8043C0B
:100CA00042F8081C0023203A02654367704700BFE2
:100CB00095020000094A0346906870B113F1160FBF
:100CC000006E05D0A0F140029A4205D8834203D2BB
:100CD000814228BF0020704700207047480900204B
:100CE00008B515460B4A0C4B9060026F1A600E4611
:100CF00000F048F82C4686F309884FF00000074BB7
:100D0000984720464FF000014FF000024FF00003DB
:100D1000034C204748090020980800206147000044
:100D200095020000014B10221A61704700ED00E0AF
:100D3000044800232021C2180133302B82F800130D
:100D4000F9D1704700E100E008B5EFF30583064AEA
:100D5000103B02EBC30152F8330049688847BDE8F5
:100D60000840FFF7E3BC00BF2C520000024B034ACF
:100D70000348012100F076B80000042000000020A4
:100D8000E4530000026E054B403A1A60044A4021C9
:100D9000C3E901121846012100F06EB89C0800203A
:100DA00000000B15084AC2F898000B6823F01F03D7
:100DB000034343F01003C2F89C308B6843F00103F7
:100DC000C2F8A030704700BF00ED00E02DE9F0430D
:100DD000DFF8608085B00E461F4604464FF00009DC
:100DE000B14523DA6068D8B13FB1411E08421BD13A
:100DF0001F2819D92368194216D12368019303F0DB
:100E0000D2FCA36803430393D8F89050C5F3072599
:100E1000D0B2013DA84207D801A9FFF7C3FF421C89
:100E200009F101090C34DBE76FF01502104605B03B
:100E3000BDE8F08300ED00E0044B0522C3F89420E8
:100E4000BFF34F8FBFF36F8F704700BF00ED00E01F
:100E5000BFF35F8F024B0022C3F89420704700BF9E
:100E600000ED00E010B5034C01232278FFF7AEFF40
:100E7000207010BD700B002008B50B4A00231278BB
:100E8000FFF7A4FF10F1160F07D0084A0021D2F88F
:100E90009030C3F30723984200DB08BDC2F89800E6
:100EA000C2F8A0100130F2E7700B002000ED00E066
:100EB0002DE9F043534B544CD3F890302568C3F3DD
:100EC00007239D4285B000F29A80FFF7C1FF002002
:100ED0000C2685421AD14D4C4D4F25706846FFF7C0
:100EE00001FBDFF82081DFF82C9106460025AE4299
:100EF00013D1237843490020D1F89020C2F3072270
:100F0000934276DBFFF798FF002042E0616806FB22
:100F10000011FFF747FF0130DBE7009800EB0511F8
:100F20004FEA051CCB683B40B3F5000F48D00AD808
:100F3000B3F5001F30D0B3F5800F36D0B3F5801F66
:100F400010D00135D3E7B3F1807F42D0B3F1007FF9
:100F5000F7D150F80C3088684A6803F024FC40F45C
:100F6000802009E050F80C3088684A6803F01BFCC8
:100F700040F0885040F43020CDE901230390D8F8A8
:100F800090302078C3F30723013B98422AD96FF0B1
:100F9000150005B0BDE8F08350F80C3088684A6849
:100FA00003F001FC40EA0900E6E750F80C308868DD
:100FB0004A6803F0F8FB40F0E06040F40030DBE703
:100FC00050F80C3088684A6803F0EDFB40F08270FE
:100FD000D2E750F80C3088684A6803F0E4FB40F030
:100FE0008870C9E701A9FFF7DDFE2378013323707C
:100FF000A7E7C1F89830C1F8A00001337CE74FF0B3
:10100000FF30C6E700ED00E0F0530000700B002059
:101010000000F0FF0000081108B50649064821F05D
:101020000701C1F1005202F5802203F044FA0020CA
:1010300008BD00BF071B0020A80800200E4A01239E
:10104000C2F840354FF080424FF08051C2F87835F9
:10105000D1F83001082808D1D1F83411052904D875
:101060000648415C09B1C2F838364FF0804301228E
:10107000C3F880250020704700E001401B570000A6
:1010800020B1034B800143F001031847704700BFB4
:10109000B05300004FF08043D3F84036DB072ED525
:1010A0004FF01023D3F8043303F00703072B26D1A6
:1010B000144A0123C2F80435D2F80034002BFBD0C7
:1010C0004FF01021D1F8043323F0070343F0040359
:1010D000C1F804330023C2F804350A4AD2F80034B8
:1010E000002BFBD0BFF34F8F0749084BCA6802F4AF
:1010F000E0621343CB60BFF34F8F00BFFDE70020DA
:10110000704700BF00E0014000ED00E00400FA0578
:10111000084B70B5C31A0D4607499B100446594346
:101120000648402203F058FB2B4601462046BDE806
:1011300070401847C8080020B76DDBB6DC510000CE
:1011400073B50C4C0C4A4023041B00930D460B4610
:101150000A49A41061430646094803F069FB011ED1
:1011600005DA30462B4602B0BDE87040184702B0A1
:1011700070BD00BFC80800209B480000B76DDBB6FB
:10118000DC51000010B5EFF31184202383F31288A3
:10119000BFF36F8F074A136823F00201DB0711606A
:1011A00002D4012003F057FD84F31188BFF36F8F41
:1011B00010BD00BF18090020002270B501210446AF
:1011C0001046FFF727FD0F4800F0F2FF0E4B984244
:1011D00015D100F0FDFF26690C49304603F021FAD5
:1011E00000280BDB012535642469084904F11C0043
:1011F00003F017FA002801DBE564002070BD6FF0F2
:101200000400FBE7091300000000AD0B10540000C0
:101210001FB500220123CDE90223094ACDF800D0F1
:101220006B46CDF804D003F031FB002805DB4FF40A
:1012300080420023684601F05DFF05B05DF804FBC5
:10124000B948000030B4104B0C2202FB00330146B9
:101250000020D3E90E529863EFF31180202484F329
:101260001288BFF36F8F1C6C04F0C00444F00204BA
:101270001C6480F31188BFF36F8F1DB12B460348A8
:1012800030BC184730BC7047C8080020DC51000053
:1012900010B4EFF31182202383F31288BFF36F8F12
:1012A0001748016841F002040460C80707D482F3BC
:1012B0001188BFF36F8F012010BC00F09BBF4FF06F
:1012C0008041D1F80C04D1F80C14C907EFD5EFF325
:1012D000118083F31288BFF36F8F0A490B6C03F000
:1012E000C00343F002030B6480F31188BFF36F8FD8
:1012F00082F31188BFF36F8F002010BCFFF7A2BFED
:1013000018090020C808002010B1012804D0704737
:10131000034B1B6C5B0701D1FFF794BF704700BF05
:10132000C80800202DE9F0413849BFF35B8F07461C
:10133000012251E8003F41E800200028F9D1BFF325
:101340005B8F33B9324933484B60CB608A6003F01E
:101350007BF97B1E012B2BD8012F07D14FF0804347
:10136000D3F81C3403F00303012B21D003F094FDC8
:101370000546F8B9284B1B78E3B14FF080430222B1
:10138000C3F808230646DFF894804FF08044D4F871
:101390001824D4F81834D20315D503F00303012B15
:1013A00001D0012F0FD155B386F31188BFF36F8F92
:1013B000BDE8F081EFF31186202383F31288BFF399
:1013C0006F8F0125DFE7ADB1304603F0DDF9D4F8CA
:1013D0001835002BDBD1D4F80421002AD7D0C4F86B
:1013E0000431D4F804310123C4F81835C8F8803129
:1013F000A360CCE70021212002F072F9E7E74FF06B
:1014000080430222C3F80423D2E700BFC4080020AF
:10141000B4080020E4080020930B002000E100E065
:10142000F0B54068057B01F01F0444EA45140569E6
:1014300087B0002D64D0B2F5001F00F1100506D171
:101440002146284603F087FC002007B0F0BD01AE1E
:101450000027B2F5800F0197776039D1B3F1007F93
:1014600014BF052304238DF804300023CDE9046361
:101470000393836823FA01F111F001011AD1B2F14B
:10148000A07F17D104F01F03620903F5E0732AD08F
:10149000012A3BD11F4A52F82330DB070AD40DF151
:1014A000030632462146284601F082F91A4B98423B
:1014B0001CD0029603AA2146284601F03BF8174BA0
:1014C000984220D101222146284601F0D5F9BBE7F8
:1014D000B3F1C06F05D0B3F1007F14BF0123022325
:1014E000C1E70323BFE74FF0A042D4E731462846C7
:1014F00001F0BCF9094B9842DBD06FF00B00A4E778
:101500006FF08500A1E76FF015009EE751F82330DA
:10151000FFDE00BF000300500400AD0B0000AD0B68
:1015200038B545682B69B3B11035284601F08EF9FE
:10153000044680B90146284601F054F9084B984208
:101540000BD108492246284601F02CF922460521F4
:101550000620FFF75FFB002038BD6FF00400FBE7BB
:101560000000AD0B69150000420970B5034602D0BA
:10157000012A17D070BD0D4E326951680029F9D08B
:1015800003F01F0301250C689D400029F2D08A68F2
:101590002A4002D04B68304698472CB12368214638
:1015A0001C46F2E7024EE7E72346F8E70452000044
:1015B000F05100002DE9F043466840F20635D006B0
:1015C000337B87B002EA050554BFC2F34010032005
:1015D00001F01F07B5F5837F144647EA43178DF8DE
:1015E000030045D00FD8062D18D007D8B5B1022D6D
:1015F00040D06FF0150007B0BDE8F083B5F5807FEF
:10160000F7D101250AE040F20222954234D0B5F527
:10161000407F33D0B5F5007FEBD1022501232203B3
:1016200003FA01F12CD57368C3F80815326982BB3F
:1016300007F01F037F0929D0012F77D13E4A02EB23
:10164000830284F48033D2F80017C3F30043C4F359
:10165000404444EA430421F4E16144EA800421F077
:10166000070144EA05230B43C2F800370020C2E714
:101670000725D3E70425D1E70525CFE70325CDE7E7
:10168000630344BF7368C3F80C15CFE74FF0A04263
:10169000D5E710360DF102023946304601F088F8E0
:1016A00014F4403F80460CD13946304603F051FBDC
:1016B000224B9845DAD19DF80210304601F0D0F85F
:1016C000D4E701AB4FF0000903AA39463046CDE913
:1016D0000439CDE90199CDF80C9000F02BFF174BA0
:1016E000984286D114F4003315D09DF803308DF85C
:1016F0000E3084F48034C4F300444B4603AA3946C8
:1017000030468DF80C508DF80D4000F0CDFF0B4B9E
:101710009842CDD06DE7CDE9043303AA0DF1030360
:1017200039463046039300F005FFF0E703F5E07318
:1017300052F82330FFDE00BF000300500000AD0B65
:101740002DE9F04FDFF8F480DFF8F490DFF8F4A033
:101750008C46002640F2FF1EF3B29C4502D80020C2
:10176000BDE8F08F50F826104F04C1F3C324C1F335
:10177000080353D4090E18F80440734508BF4FF00E
:10178000FF3303294DD8DFE801F002083033C2F8F7
:101790000C35591C2FD10136DEE7C2F814355D1C1B
:1017A000F9D0002550F8261001F40047002F16BF8D
:1017B0000025AB464FF0010B03F01F075B092AD051
:1017C000012B35D1534603EB8707C1F34121240296
:1017D000D7F8003744EA81042C4303EA090344EABA
:1017E0004B042343C7F80037D5E7C2F80835D0E7E4
:1017F000C2F81035D3E759090AD0012914D1114F85
:1018000003F01F01012505FA01F1C7F80815C9E722
:101810004FF0A047F4E74FF0A043D4E76FF0150076
:101820009EE76FF085009BE70023C3F80835FFDED5
:1018300007F5E077002353F82730F8E74C5700000E
:10184000F0F8FCFF000300502DE9F0410446476822
:101850000D4603F021FB4FF0200888B9264B1B787A
:1018600073B16426606803F036F9F0B9012003F023
:10187000E4F9013EF6D10021212001F031FFF0E72B
:10188000EFF31186314688F31288BFF36F8F6068DB
:1018900003F021F9A8B986F31188BFF36F8FEFE742
:1018A00086F31188BFF36F8FE5E7EFF311863146BA
:1018B00088F31288BFF36F8F606803F00CF900287B
:1018C000EED0BB691D706368BA691B680020C3F85D
:1018D00044250122C3F84825C3F82001D3F820414C
:1018E000C3F85801D3F858019A6081F31188BFF307
:1018F0006F8FBDE8F08100BF930B0020F7B5054660
:10190000002201210220FFF785F90220FFF766F986
:101910006A6811681369C1F82435137D507D927D82
:1019200003431343C1F86C356E68D6E9004313F0E6
:10193000010348D02F6907F10C0003F08AF9304BFE
:1019400098425AD1387B04F10C0204F5907103F0EF
:1019500076F9387B012707FA00F000F0C1FB082375
:10196000C4F80035B369C4F844350023C4F84835D9
:10197000A760D4F85831002BFBD00021C4F8001523
:101980006B68DC6801AA204602F0EEFF002805DB48
:10199000019B226819791868FFF7D2FE6A681368FC
:1019A0000821C3F80015117A51B9D269C3F834255A
:1019B0000122C3F83825C3F81011D3F810111A60AA
:1019C000002003B0F0BD0822C4F80025B269C4F8B5
:1019D0004425C4F848350123A360D4F82031002BF6
:1019E000FBD00023C4F82031D4F820310123E36078
:1019F0004FF48073C4F80433BBE76FF00400E0E7F2
:101A00000000AD0B70B5012383400E4ABFF35B8F1E
:101A1000DC4352E8001F01EA040542E80056002EAC
:101A2000F7D1BFF35B8F4FF4803282400648C0F895
:101A30000823BFF35F8FBFF36F8F0B4214BF0120EA
:101A4000002070BD380900200010014070B40E491C
:101A5000D1E90034D01AC31844F1000422F07F46C3
:101A6000C1E90034A6F50013B3F5400F09D2074BC6
:101A70001B681A0A1B069C19054B42F10005C3E9B5
:101A8000004570BC01F0B0BFC80100203C09002037
:101A9000D001002011B3BFF35B8F0123104A8340B4
:101AA00052E800CF4CEA030C42E800C10029F7D10C
:101AB000BFF35B8F0B4A4FF480338340C2F804338B
:101AC000094BBFF35B8F1B68BFF35B8FC340DB0722
:101AD00042BF064B4FF40032C3F80021704700BFED
:101AE00038090020001001403409002000E100E026
:101AF0000D4B1868010A0006BFF35F8F0B4BD3F83C
:101B00000435181841F10001B3F5801F0AD2084BC3
:101B1000D3E90023904271EB030303D210F18070EC
:101B200041F10001704700BF3C0900200010014056
:101B3000D00100202DE9F04F85B016461F469DF8D4
:101B400040A00446FFF75EFF0190FFF7D1FFB042CF
:101B500071EB070354D23E4B301A67EB01019842F8
:101B600071F100014FD23B4B03EB0413D3E9022385
:101B70009F4208BF96425ED037494FF4803804F147
:101B8000500508FA04F8AD00C1F848832046ADB20C
:101B900003F03BF826F07F4B05F1804504F5A87370
:101BA00005F58835DC464FF003090293029A2CF0C4
:101BB0007F4341F82230C1F84483D1F80435274AE5
:101BC0006FF00200C01A604420F07F40904232D98A
:101BD000286868B1D1F804350393A3EB0B0020F01B
:101BE0007F40B0F5000F26D9204603F00EF8039B86
:101BF000BAF1000F07D109EB030C09F10109D5E790
:101C0000BAF1000F09D06FF0150520460199FFF7D2
:101C100041FF284605B0BDE8F08F0123104ABFF30D
:101C20005B8FA34052E8000F184342E800010029EF
:101C3000F8D1BFF35B8F07490E98230101EB041223
:101C4000C8500F9B5360C2E902670025DDE700BF63
:101C500001008000B801002000100140FDFF7F005E
:101C6000340900207FB51C4C1C4BC4F80833C4F861
:101C700048331B4B00254FF0FF304FF0FF31C4F8C5
:101C80000855C3E902014FF48033C4F80433154BFF
:101C900002264FF400320121C4F804631120C3F876
:101CA00080212A46FEF7B6FF1120FEF797FF0E4A65
:101CB0000123A360236013600C4B0D4A0093CDE910
:101CC000015500232846FFF735FF3046FFF72AFB72
:101CD000284604B070BD00BF0010014003000F0093
:101CE000B801002000E100E0380900204D1A000092
:101CF000FFFF7F002DE9F7432F4CD4F804339907F9
:101D00000BD5D4F8043143B12C4A0023C4F8043174
:101D1000D4F80431136801331360D4F80433DA03C0
:101D200029D5BFF35B8F264B53E8002F22F001012A
:101D300043E800100028F7D1BFF35B8FD30702D42C
:101D4000D4F84031BBB10025C4F84051D4F840313B
:101D5000FFF7CEFEEFF31182202383F31288BFF347
:101D60006F8F184BD3E90267B042B94106D282F3B4
:101D70001188BFF36F8F03B0BDE8F0834FF0FF38D9
:101D80004FF0FF39C3E90289D3E900101D604FF419
:101D90008033C4F84833C4F84051D4F8403182F35A
:101DA0001188BFF36F8F0029E5D0009032463B4683
:101DB00028468847DFE700BF001001403C090020AB
:101DC00034090020B801002030B5431C124C85B006
:101DD00005D08442A8BF0446012CB8BF0124FFF7F8
:101DE00087FE0E4B0C4DD3E90013401AB0F5000FDF
:101DF00010D22218AA4228BF2A4652184FF00000DB
:101E000007490091CDE9010043F10003FFF792FE7D
:101E100005B030BD2A46F0E7FFFF7F00C801002073
:101E20004D1A000008B5FFF763FE024B1B68C01A8D
:101E300008BD00BFC8010020BFF34F8F0549064B06
:101E4000CA6802F4E0621343CB60BFF34F8F00BF58
:101E5000FDE700BF00ED00E00400FA054FF08053FD
:101E6000D3F83021082A06D1D3F83431052B02D813
:101E7000024AD05C70470020704700BF68570000DE
:101E8000024AD2F80034002BFBD0704700E001403A
:101E900010B54FF08053D3F83021082A4ED14FF0BF
:101EA00080420021C2F80C11C2F81011C2F8381596
:101EB00002F54042D3F80414C2F82015D3F80814F0
:101EC000C2F82415D3F80C14C2F82815D3F810144E
:101ED000C2F82C15D3F81414C2F83015D3F818141E
:101EE000C2F83415D3F81C14C2F84015D3F82014E6
:101EF000C2F84415D3F82414C2F84815D3F82814AE
:101F0000C2F84C15D3F82C14C2F85015D3F830147D
:101F1000C2F85415D3F83414C2F86015D3F8381445
:101F2000C2F86415D3F83C14C2F86815D3F840140D
:101F3000C2F86C15D3F84434C2F87035FFF78EFF41
:101F400018B13F4B3F4AC3F88C26FFF787FF18B103
:101F50003D4BFB22C3F81825FFF780FF70B14FF00F
:101F600080414FF08053D1F8E42ED3F8583222F05C
:101F70000F0203F00F031343C1F8E43EFFF76EFFB7
:101F800020B1324B4FF40072C3F840264FF080531B
:101F9000D3F83031082B1AD14FF08043D3F8002406
:101FA000D20744BF6FF00102C3F800244FF0805302
:101FB000D3F83431052B02D8254AD35C3BB14FF01E
:101FC0001023D3F808224FF08043C3F858254FF070
:101FD0001021D1F80C32DB0714D51E480123C0F8BC
:101FE0000435FFF74DFFD1F80C3223F00103C1F89F
:101FF0000C32FFF745FF0023C0F80435FFF740FF20
:10200000FFF71AFFD1F80032002B03DBD1F80432BE
:10201000002B14DA0F4901234FF01020C1F80435CA
:102020001224FFF72DFFC0F80042FFF729FFC0F888
:102030000442FFF725FF0023C1F80435DEE710BD99
:10204000005000404881030000F000400090024032
:102050006257000000E0014030B50468CCB1BFF326
:102060005B8FB4FA84F3C3F11F03DBB201229A4001
:1020700024EA020250E8005FA54204D140E8002CA7
:10208000BCF1000FF6D1BFF35B8FE6D102480B70B5
:1020900030BD0248FCE700BF0000AD0B0200AD0BF5
:1020A00010B50368CB40DB0714D401238B400268D2
:1020B000BFF35B8F43EA020150E8004F944204D122
:1020C00040E8001CBCF1000FF6D1BFF35B8FEED1EE
:1020D000014810BD0148FCE70000AD0B0400AD0B4A
:1020E000014BC3F80405704700F00140F7B5044602
:1020F00018B1012823D003B0F0BD4FF08043022275
:10210000C3F808230122DA60C3F80401D3F80431CC
:10211000064601238DF8073042F210754FF08047D4
:10212000D4B1012CE7D1D7F80C3403F48033AEBB23
:1021300083B3012002F081FD013DF4D12AE04FF08C
:1021400080430022C3F808035860C3F80021D3F885
:1021500000310DF10706DCE7D7F8183403F48033BB
:102160003EB9002BC7D0012002F067FD013DF3D13D
:10217000C1E7D7F8182402F003023260002BBAD06E
:102180009DF80700012803D102F057FD013DC7D19A
:10219000012CB0D1054B00225A71ACE7D7F80C24C2
:1021A00002F001023270002BEAD1F3E7400900206F
:1021B000044B1A7922B9012218609A8002487047AC
:1021C00002487047400900200000AD0B0C00AD0B29
:1021D00008B5074B1B682BB10020FEF70DFD08B9B1
:1021E000FEF7FCFC4FF080430022C3F8182508BD21
:1021F0004009002010B510B1012843D010BD4FF0A8
:102200008043D3F81814D3F81824C80321D502F05A
:102210000303012B04D013B10020FFF767FF002355
:102220004FF080420220C2F8183508224FF4827322
:1022300003F180430021196002F180421C680124EF
:102240001460154A12680AB34FF08043C3F80403C0
:10225000D4E7D3F81424D107E1D5D3F81C2492078E
:10226000DAD40D4A12681AB10222C3F80423C5E772
:10227000D3F80421002AFBD00022C3F80421D3F8AC
:102280000431BBE700224FF48073D1E71A68002ABB
:10229000FCD019601B68B1E74009002010B54FF071
:1022A0008043D3F800216AB10022C3F80021D3F89B
:1022B00000210122C3F80823114B587910B95A7133
:1022C0001B6898474FF08043D3F8042172B1002275
:1022D000C3F80421D3F80421D3F81824D3F8182420
:1022E000920704D10122C3F818259A6010BD02227A
:1022F000C3F80823024BBDE810401B6801201847B3
:1023000040090020036803F01F025B09026004D04B
:10231000012B034818BF002070474FF0A0407047C2
:1023200000030050034A430900F01F00D35C184427
:10233000C0B270476E57000070B50546FFF7F2FF58
:102340000C4C08300E4634F81030DA0508D5C3F3CB
:10235000432304EBC302284654F8333052689847AD
:10236000A3682BB1E26831462846BDE870401847A3
:1023700070BD00BF4800002008B5FFF7D3FF034B36
:10238000083033F81000400B08BD00BF48000020A3
:1023900008B5FFF7C7FF034B083033F81000C0F350
:1023A000400008BD4800002008B5FFF7BBFF034B05
:1023B000083033F81000C0F3401008BD480000207A
:1023C000034611F0010010B5CCB20DD1A207C4F341
:1023D000400012D5094AD2F820055860C2F82005FD
:1023E000003818BF012008E04FF0A041D1F82025A7
:1023F0001A60C1F82025002AE8D010BD0003005063
:1024000010B5FFF78FFF124A083032F81030D905A7
:102410001CD5C3F3432123F4F85322F8103002F102
:102420000E04002034F8023F13F4807F03D0C3F37E
:10243000432399420AD001303028F3D1002342F8D7
:1024400031300448BDE81040FFF72ABE10BD00BF80
:1024500048000020C0000020F0B5054600200446DA
:10246000012607468C420BD1114BD3F87C2132B1A7
:102470000022C3F87C21D3F87C3140F00040F0BD4D
:10248000E3B29B0003F580729B0806FA03F31D423A
:102490000BD002F1804202F5C042D2F800C0BCF17C
:1024A000000F02D01760126818430134DAE700BF4A
:1024B00000600040F7B506460846FFF733FF194FA6
:1024C00000F108050C4637F81530DB0727D53046F4
:1024D00002F01BFC2046FFF767FF40B12046FFF7E4
:1024E0004BFF316800F5A270002341F820302046F0
:1024F000FFF786FF002301A827F815300194FFF7A6
:1025000001FF019B00EB8300074BD0F8002713402D
:1025100043F00203C0F80037044803B0F0BD04489C
:10252000FBE700BF48000020F0F8FCFF0000AD0B07
:102530000400AD0B2DE9FF41164680460846FFF723
:10254000F1FE0D463168044609B32846FFF720FF27
:1025500018B12846FFF728FF10BB0023CDE9003350
:102560008DF80E308DF80F300DF10F020B46284616
:102570000DF10E0102F071FB474A04F1080132F837
:10258000113023F0020343F0010322F81130736885
:1025900063B328461F785968FFF7FAFE10B1D1B12E
:1025A0003E4826E03C4A04F1080032F8103023F09F
:1025B0002003DB04DB0C22F8103061B1032FEFD8CD
:1025C0007168496891F800C0D8F80010A7B90CF5F7
:1025D000A27C41F82C70304A04F1080132F8113025
:1025E00023F01C0343EA870322F81130B3684BBB86
:1025F0002B4804B0BDE8F08101EB8C0143EA4C3379
:10260000D1F810E52EF0030EC1F810E5D8F800104F
:1026100001EB8C0E43F02003DEF8101522F8103089
:1026200021F44F3121F44071CEF810152902DEF863
:10263000108501F47C5141EA074141EA0801CEF8D6
:102640001015C8E7D3E900672846FFF7D9FE002E2A
:10265000CED0114DD5E90023964203D19F4201D13E
:10266000002209E00F480DF10F01FFF7F5FC0C4BBC
:102670009842BED19DF80F2045F8326005EBC203A9
:1026800008345F6035F8143043EA422343F4807322
:1026900025F81430ACE700BF480000200400AD0B63
:1026A0000000AD0BC00000202DE9F0430C4685B0C2
:1026B0008046204611461E46FFF734FE054629B3E4
:1026C0002046FFF765FE18B92046FFF76DFE18BBE0
:1026D000314F05F1080937F8193013F01C0F02D0FB
:1026E0004B78012B18D001238DF80F300023CDE952
:1026F00000134A1C8B1C20460DF10F0102F0ADFAAD
:1027000037F8193043F0030327F81930002E41D071
:102710002046FFF73DFE18B9204805B0BDE8F0831C
:1027200096F800C0D8F800301B4F0CF5A2720021BB
:1027300043F8221005F1080237F8121021F02001A9
:10274000C904C90C27F8121075781DB3D8F8000019
:10275000B67800EB8C002D04D0F8103523F49913D3
:1027600023F4F853C0F81035230203F47C5305F426
:1027700040353605D0F810E52B4306F4801641EAC3
:102780004C31334341F0200143EA0E0327F8121085
:10279000C0F810350248C0E7480000200400AD0B27
:1027A0000000AD0B014BC3E9021270474800002046
:1027B00010B508461446FFF7F7FD50B10846FFF77D
:1027C000B1FD054B083033F8103004485B0B237023
:1027D00010BD0348FCE700BF480000200000AD0B1F
:1027E0000400AD0B70B5164D95F8804006462CBB25
:1027F0002146602205F1100002F04AFC30682E6F7D
:1028000021468E420ED10023C0F87C31D0F87C31B5
:1028100040F30730FEF7E2F901230A4885F88030DB
:10282000AB6770BDCBB29B0003F580727C2B08BFF9
:10283000845001F1010108BF8358E2E70248F0E744
:10284000480000200000AD0B0C00AD0B034B93F8CB
:102850008000003818BF0120704700BF48000020EA
:102860000148FFF71DBC00BFBC0000200148FFF776
:10287000F3BB00BFBC00002073B503681646D3F855
:102880000423002AA8BF4FF000420546A8BFC3F8A2
:10289000042308460C46FFF787FD00B30846FFF700
:1028A00077FD0146D8B92046FFF766FD04B2A400C3
:1028B00004F58072034628688150296882582144B3
:1028C000D1F8102542F00102C1F810252EB1296877
:1028D000012202FA03F3C1F8043302B070BD2046AE
:1028E000FFF720FD0F4B083033F81030C3F382039D
:1028F000042B12D0052B12D001A80194FFF702FD82
:10290000019AD0F81035D34003F00103991C2046FA
:1029100002B0BDE8704002F0E9B90321F7E70221F7
:10292000F5E700BF480000202DE9F04F694BDFF8C4
:10293000A881D3F80403D8F87010C0B289B040F071
:102940000040FFF789FD051E2FDAC24600235AF822
:102950007C1F06A8CDE90633FFF732FD5F4B0193DC
:102960000DF118094FF0000B019A12F8013B01928A
:10297000DA0803F007031AF8022022FA03F3DA0751
:102980001CD409F10409BBF1000F14D0D8F8701061
:102990004FF00040FFF760FDD8F87C1006A8FFF765
:1029A0000FFD0028DAD125F000450124002D79D152
:1029B00009B0BDE8F08F4FF0010BD5E7484B5B4401
:1029C0000293D9F800100029DBD0029B91FAA1F103
:1029D0001C78B1FA81F141EA44142046FFF7A2FCC9
:1029E0000830059438F81070C808BB0819F80020A2
:1029F000039301F00701012303FA01F122EA010226
:102A000009F8002005A8FFF77DFC059A039B02F555
:102A1000E072C7F3820650F822205B073746C2F304
:102A2000014224D520463946D6B2FFF785FC05A8D9
:102A30000594FFF767FC059B03F5E07350F823301E
:102A4000C3F301439E4207D10021204602F04EF914
:102A50003146204602F04AF905A80594FFF752FCDA
:102A6000059B012202FA03F3C0F82035A9E7022AE8
:102A70000CD10321204602F039F906F00503012BA1
:102A8000EAD139462046FFF757FCE5E70221204608
:102A9000039202F02BF9032EF3D0039A032ADBD121
:102AA000022EEDE795FAA5F3B3FA83F304FA03F2E5
:102AB0009B0003F1804303F5C04325EA0205D3F8E8
:102AC0001005D3F81015C0F30520C1F30141FFF73D
:102AD00033FC6BE700600040480000207E57000098
:102AE0007E57000001460148FFF7B6BACC0000202F
:102AF00038B5EFF31185202383F31288BFF36F8F6E
:102B0000064B9C6802F041F985F31188BFF36F8F83
:102B10002046BDE83840FDF7E5BF00BF480900206A
:102B200038B5094B53F82040013053F82050A542E6
:102B300000D838BD636823B1204602F029F9083473
:102B4000F5E723689847FAE72455000070B52B4B4A
:102B50002B4C2C4D012286B003201A70FFF7E0FFAA
:102B6000FDF7C6FC02F030F90420FFF7D9FF264636
:102B7000AE4204F1300410D300F0F4FC204C224E9D
:102B8000AC4226D300F002FDFDF71AFB1F4A137B6F
:102B900023F00103137306B070BD54F80C3C059389
:102BA00054F8103C049354F8143C039354F8183C24
:102BB000029354F81C3C019354F8203C009354E9D0
:102BC0000A2354E90C0100F0BBFA54F8303C5E656E
:102BD000CDE7D4E90A23B3F1FF3F08BFB2F1FF3FCD
:102BE00005D052EA0301206803D102F05BF93034CA
:102BF000C6E73146183000F07DFEF8E7930B002061
:102C0000AC530000AC530000B14F0000580200204C
:102C100008B50348034A0021121A02F0D1F808BD92
:102C2000B8010020980B002070B5002386B0012267
:102C3000CDE90423134E144D01930F22CDE9023246
:102C40001249142303FB005506EBC01604464FF44B
:102C5000C07000FB04110E4B00954FF4A07230467B
:102C600000F06EFA737B0B4AEE6023F0040373737B
:102C70004FF4046304FB033313442C746B6006B0FD
:102C800070BD00BFD80100204809002000140020BA
:102C9000654E0000C00B0020BFB50020FFF740FFCD
:102CA0002C4B83F308882C4D2C4E6B692C4F43F42E
:102CB00000736B610024E02385F82230EC772C76DA
:102CC0006C76AC7685F820406B6A43F4E0236B6247
:102CD00085F82340FDF782FEFEF724F84FF0FF331E
:102CE000AB62EB62FEF7E4F8FEF740F81D4BB36011
:102CF00040F201129A81C3E91844DC6602F031F80F
:102D00000120FFF70DFF0220174DFFF709FF00F02C
:102D10005DFC164B75610593012315490094CDE9BF
:102D200003434FF480623B46CDE90144284600F05E
:102D300007FA6A7B064622F0040228466A7302F00C
:102D4000EDF82046FFF770FF3A4631462846FDF77A
:102D5000C7FF00BF0014002000ED00E0480900207C
:102D60004D2B0000D80200205802002080570000A0
:102D70008015002038B5064C064D0020AC4200D32B
:102D800038BD204602F021F80028F9DB1C34F5E7B5
:102D9000400100204001002073B50C46EFF3118183
:102DA000202585F31288BFF36F8FC5685DB125605C
:102DB0002B68C360836901338361002081F311882C
:102DC000BFF36F8F11E052EA030603D125606FF065
:102DD0000B00F3E7CDE900230246083000F00EFBBC
:102DE00018B9034B9B685B69236002B070BD00BFDC
:102DF000480900202DE9F34104460E4600F1080879
:102E0000EFF31187202181F31288BFF36F8F056ADA
:102E1000C1688D422AD202F0CFF8A2680546314639
:102E200078B10024406902F025F92846AC6702F029
:102E300075F84046394600F051FB204602B0BDE827
:102E4000F081E06902F016F9E369A268134462694F
:102E5000E361934204BF2369E361236A0133236280
:102E6000002087F31188BFF36F8FE7E752EA030171
:102E70000AD0074989684E61CDE9002339460246E8
:102E8000404600F0BBFAD9E76FF02200E9E700BF47
:102E900048090020F7B5044604F108070846EFF397
:102EA0001186202181F31288BFF36F8F216A0029D8
:102EB00031D0A268A16902F0DDF8A369A2681344C9
:102EC0006269A361934204BF2369A361236A013B42
:102ED0002362204602F070F8054660B34169A2689B
:102EE000E06902F0C7F8E369A26813446269E3612C
:102EF000934204BF2369E361236A01332362002400
:102F00002846AC6702F00AF83846314600F0E6FA87
:102F1000204603B0F0BD52EA03010AD0084989688F
:102F20004861CDE9002331462246384600F066FA72
:102F3000EFE76FF0220086F31188BFF36F8FE8E7A9
:102F4000480900202DE9F341044617461E46EFF3D9
:102F50001188202383F31288BFF36F8FC368334A2D
:102F60007BB180689168884219D057EA060318D16E
:102F700088F31188BFF36F8F6FF00F0002B0BDE8C8
:102F8000F081916891F90E1021610133E36093683B
:102F9000A36088F31188BFF36F8F0020EEE72169EB
:102FA000F2E791F90E1090F90E309942A8BF194638
:102FB0006FF07E029142B8BF11468B422DDD01F0C9
:102FC0005CFF0546CDE9007619482246414600F0EF
:102FD00015FA0028E1D0EFF31186202383F312883D
:102FE000BFF36F8FA068D0B1236821699C420AD0DB
:102FF0004BB193F90E309942A8BF19466FF07E038A
:103000009942B8BF194601F038FF40B1084831462F
:1030100000F064FA6FF00A00B0E70025D2E7002D57
:10302000F4D186F31188BFF36F8FF3E748090020CE
:10303000940B002038B58368044663B3194A92683C
:1030400093422BD1C368012B03D9013BC3600020FD
:1030500038BDEFF31185202383F31288BFF36F8F00
:103060000169806801F009FF204601F0A5FFA0601A
:1030700058B190F90E2022610022826701F04EFFC4
:103080000948294600F02AFAE1E7E06085F3118853
:10309000BFF36F8FDBE76FF01500D9E74FF0FF301C
:1030A000D6E700BF48090020940B002038B504463D
:1030B000EFF31185202383F31288BFF36F8F01F0A4
:1030C0007BFF48B10022826701F028FF29460848AB
:1030D000BDE8384000F002BAD4E902329A4218BF83
:1030E0000133A36085F31188BFF36F8F38BD00BF34
:1030F000940B002013B5EFF31181202484F3128880
:10310000BFF36F8F846844B1013C846081F3118800
:10311000BFF36F8F002002B010BD52EA030406D146
:1031200081F31188BFF36F8F6FF00F00F3E7CDE9E4
:1031300000230246014800F061F9ECE7940B0020FF
:103140002DE9F043073285B022F007020E461F46F4
:103150001099017300F158037F32C0E91633044619
:10316000002322F03F020421836041733F2A0F981D
:10317000A073C4E90633E37306F14009A2F14008E5
:1031800005D883F31188BFF36F8F084602DFB518A7
:1031900029462046FDF7AAFA07300E9B20F00700CB
:1031A000A066C4E9189802930D9B01932D1A0C9BFD
:1031B00000932A463B4631462046FDF75FFD00233B
:1031C0006365044B9B6803B1DB6EE366284605B07C
:1031D000BDE8F0834809002038B50D4D2B4653F863
:1031E000184F9C4200D004B9EC68AB6838B95A7BE0
:1031F000D20604D1A26912B9DA897F2A05D89C4285
:1032000002D0204600F0BEFA23466B6138BD00BFF5
:103210004809002008B590F90D20437B002A01469B
:1032200004DA03F07F03437301F03EFE044B986819
:10323000431A58425841BDE80840FFF7CDBF00BFD0
:103240004809002070B490F90D30427B002B29DB37
:10325000D30627D183692BBB134962F07F024273E7
:103260000A4652F8184F944218BF2346CC6923B936
:10327000C0E900242060C8610CE090F90E5093F979
:103280000E60B5420AD0AE4208DD5A68C0E900328D
:103290001060586070BC0020FFF79EBF9C42E7D0D2
:1032A0001B68E4E770BC7047480900202DE9F04135
:1032B000002A427B0E460CBF102108211142044611
:1032C0000FD141EA0203D20918D1437308291BD058
:1032D0000120FFF781FFBFF35F8F637B23F0600363
:1032E0006373274B9B68A34243D1EFF30583002B05
:1032F0003FD13046BDE8F041FDF70ABC03F07F0343
:10330000437301F0D1FDE1E7A36813B1204601F05A
:10331000D3FD04F1180001F08CFEA56D04F15807EF
:10332000AF4211D04FF0000875B1284601F0C4FD3E
:1033300005F1180001F07DFEC5F878802846FFF7FA
:1033400081FFA56DAF42EFD10D4DAB689C42BFD15F
:10335000EFF30583002BBBD00120FFF73DFF094BA6
:10336000AB6040F201129A810022C3E91822DA66AA
:10337000B1E786F31188BFF36F8FBDE8F08100BF1E
:1033800048090020D802002070B590F90D20437B39
:10339000002A014604DA03F07F03437301F084FD41
:1033A0004B7B154A63F07F0310464B7350F8183F70
:1033B000D469834208BF002323B9C1E90004216016
:1033C000D1610CE091F90E5093F90E60B5420ED028
:1033D000AE420CDD5868C1E9003001605960906868
:1033E000431A5842BDE870405841FFF7F5BE9C4271
:1033F000E3D01B68E0E700BF48090020F8B5124B96
:103400000C461146114A98681060DDE90676EFF324
:103410001182202282F31288BFF36F8F9D682846A5
:1034200001F054FDB6F1FF3F08BFB7F1FF3F06D0F2
:1034300007493A46334605F1180000F05BFA20468A
:10344000BDE8F840FDF764BB48090020680900208A
:10345000B14F0000F8B50446EFF31186202383F343
:103460001288BFF36F8F437BDA0649B219D18569A1
:10347000BDB903F07F03437301F016FD437B164A89
:10348000817363F07F034373134653F8180F984218
:1034900018BF0546D0695DB9C4E900300460D46145
:1034A00011E0A173002086F31188BFF36F8FF8BD80
:1034B00095F90E70B9420BD08F4209DD6B68C4E9F3
:1034C00000531C606C600120FFF786FE0120EAE7D4
:1034D000A842E1D02D68DEE74809002049B9EFF3A2
:1034E000058030B9054B5A699B689A4201D0FDF7B7
:1034F0000FBB81F31188BFF36F8F7047480900201D
:1035000010B5EFF31184202282F31288BFF36F8F7E
:10351000427B510704D484F31188BFF36F8F10BD31
:1035200022F004024273FFF78DFE21460248BDE8F7
:103530001040FFF7D3BF00BF940B0020034648B9EB
:10354000EFF3058232B9064A51699268914201D07F
:10355000FDF7DEBA83F31188BFF36F8F704700BFAA
:1035600048090020EFF31181202383F31288BFF371
:103570006F8F054B9A68D37B013BD37381F311881E
:10358000BFF36F8F704700BF4809002038B5EFF3D5
:103590001185202484F31288BFF36F8F0A4B9A6839
:1035A000D37B0133D3730020FFF716FE85F3118818
:1035B000BFF36F8FEFF3118084F31288BFF36F8F27
:1035C000BDE83840FFF7BABF48090020024B03F1BD
:1035D0001802C3E90622704748090020F8B5EFF346
:1035E0001185202383F31288BFF36F8F19498868F0
:1035F000437B03F07F03437301F056FC8B685A7BD7
:10360000084662F07F025A7350F8182FCC69824244
:1036100008BF002222B9C3E900042360CB610CE09B
:1036200093F90E6092F90E70BE420ED0B7420CDDD7
:103630005168C3E900210B6053600120FFF7CCFD06
:103640002846BDE8F840FDF763BAA242E3D012680D
:10365000E0E700BF4809002050EA01032DE9F041EE
:1036600005460E4603D1FFF7B9FF00202BE0831C6F
:1036700071F1FF3329DB01F0F1FC2C18EFF3118815
:10368000202383F31288BFF36F8F124F124BB86859
:103690001860FFF7BFFDB86810492A463346183056
:1036A00000F028F9BA68537B43F010035373404687
:1036B000FDF72EFA01F0D2FC201A63EB0303012878
:1036C00073F10003D1DBBDE8F0816FF00104241A2F
:1036D000D4E700BF4809002068090020B14F00006E
:1036E000B1F1FF3F08BFB0F1FF3F08B506D10A4B6B
:1036F000986801F022FC4FF0FF3008BDFFF7ACFFE7
:103700004FF47A7147F6FF730022C0FB0132D80BE9
:1037100040EA4240F1E700BF48090020014B9868A9
:10372000704700BF48090020044BC01A044BC0106A
:103730005843044B01221A54704700BF580300201D
:10374000ABAAAAAA940B0020C3897F2B12D80A4BDC
:103750001B6863B1094B90F90E201B689A4209DB84
:10376000437BDB0606D1064BC31A18BF012303F0C7
:10377000010070470023FAE7700900206C0900205F
:10378000D801002070B50E4B0E4C1E7C06EB460394
:1037900004EBC3040546204601F04BFC0A4B002213
:1037A00028469A55FFF7D0FF48B1084B08491A68D8
:1037B000013A2046D317BDE8704000F09BB870BDB9
:1037C0004809002058030020940B002070090020B5
:1037D0002937000038B5EFF31185202383F31288D1
:1037E000BFF36F8F104B114A9C681068A04206D13E
:1037F000FFF7C8FF85F31188BFF36F8F38BD002135
:103800001B7C11600A4AD35C002BF3D02046FFF7E3
:103810009BFF0028EED0637BDB0602D12046FFF73A
:10382000B3FD2046E4E700BF4809002068090020F6
:10383000940B002008B50648064A0749121A01F001
:10384000C1FABDE80840054A0549064801F0BABA80
:1038500000000020B8010020945700000000000084
:103860009457000000000020034B1B680BB9FEF7C3
:10387000D9BA0020704700BF7409002030B570B17C
:103880000B4B5B6898420AD0036843B1D3E904212B
:10389000D0E90445121941EB0501C3E90421D0E93F
:1038A000003213605A600023C0E9003330BD00BF0E
:1038B000D000002010B50E4B1C689C4204D1FFF7CD
:1038C000D3FF6FF0004010BDFFF7CEFF002CF8D003
:1038D000D4E904321B1A62EBE072B3F1004F72F1CB
:1038E0000001EEDA002AACBF18460020EBE700BF6B
:1038F000D0000020B3F1FF3F08BFB2F1FF3FF8B5A1
:1039000004461D4616465ED08160EFF311872023E2
:1039100083F31288BFF36F8F013275F1FF3324DA1E
:103920002E49D1E900206FF001039B1A4FF0FF32BE
:1039300062EB00009E1B60EB0500012E70F100039E
:1039400001DA01260020C4E90460254ED6F800C043
:103950007568B44508BF4FF0000CBCF1000F0DD1E5
:10396000C4E900652C6074601CE0FFF77DFF013640
:1039700045F10005361845EBE070E4E7DCE904208A
:10398000D4E90431934271EB000E1DDAD21ADCF84F
:10399000043060EB0100CCE90420C4E900C31C60E2
:1039A000CCF804403368B34209D09C4207D10D4B98
:1039B0001C6824B9FFF77EFF2146FEF705FA87F35E
:1039C0001188BFF36F8FF8BD9B1A61EB0001AC4506
:1039D000C4E90431C4D0DCF800C0BEE770030020A5
:1039E000D0000020740900202DE9F84FEFF3118C6E
:1039F000202383F31288BFF36F8FDFF8B0A0DFF8C6
:103A0000B0902C4FC9F80000DAF8000000245045AF
:103A100008BF00200025D7E90021D9F80030E04692
:103A200078B3D0E9046C4FEAE37EB3427EEB0C0B33
:103A300005DAF61A6CEB0E04C0E9046421E0B21852
:103A400041EBE671C0E90445C7E90021FFF716FF25
:103A500088F31188BFF36F8F83689847EFF311885D
:103A6000202383F31288BFF36F8FD9F80030DAF880
:103A700000009B1B5045C446C9F80030CBD1D7E9A4
:103A800000219A1841EBE3730024C7E90023C9F829
:103A90000040FFF70FFF2146FEF796F988F31188E3
:103AA000BFF36F8FBDE8F84FFFF794BED000002042
:103AB000740900207003002010B5EFF31184202357
:103AC00083F31288BFF36F8FFFF7CEFE054A0346DC
:103AD000D2E90001181841EBE37184F31188BFF3B8
:103AE0006F8F10BD7003002038B5064C064DAC42F8
:103AF00001D3002038BDD4E90112204601F0B2FA0A
:103B00001434F4E7400100204001002010B50A4CB5
:103B100023681BB101232360002010BD00F0EAF8E8
:103B20000028F7D00138062803D8044B53F82000AA
:103B300010BD034810BD00BF780900203C550000AF
:103B4000FE8FFFFFBFF34F8F0549064BCA6802F493
:103B5000E0621343CB60BFF34F8F00BFFDE700BFB0
:103B600000ED00E00400FA0510B4094B09490A4CC5
:103B70004FF0FE32C3F800244968C3F80424C3F8A8
:103B80000824C3F80C240023C4F8003510BC0847EF
:103B900000B00250D800002000A00250D0E900126E
:103BA000014BC3E900127047D800002010B504464D
:103BB00050B1636813F0685F05D0064A934202D0A3
:103BC00000232360626010BD034B04485B68984784
:103BD000EFE700BF2C5F5CA9D8000020585500001B
:103BE000C8B143680D4A934213D013F0685F0ED0FA
:103BF000012350E8002F194640E8001C9CF0000FFC
:103C0000F7D1012AF5D0BFF35F8F00207047044839
:103C10007047044870476FF4E04070472C5F5CA920
:103C2000E98FFFFFEA8FFFFF80B14368094A9342A3
:103C30000AD013F0685F05D0BFF35F8F00230360E5
:103C40001846704704487047044870476FF4E040D6
:103C5000704700BF2C5F5CA9E98FFFFFEA8FFFFF71
:103C600010B5044620B1044B63600022226010BDF1
:103C70000248FFF779FFF6E73A00003A8055000066
:103C800070B5D0E90023174C174D6360D0E90230BE
:103C9000C4E9023022604868D1F800C0134BC3E980
:103CA00000C0D5F81801D1F808C0C3F808C010F05A
:103CB000685FD1F80CC00969C3F80CC0196110D055
:103CC0000B49C5F8BC110023C5E9453105F58A70DB
:103CD000C5F8B8319047236805F5DC70BDE8704041
:103CE000184770BDF400002090090020E00000207B
:103CF0002C5F5CA938B500F02FF820B1032400F048
:103D000063F8204638BD00F031F898B900F0ACF8FF
:103D100098B90F4DD5F828391B0EF02B08D1D5F8DE
:103D2000242A0C4B9A420AD0072400F017F8E6E741
:103D30000624FAE70424204638BD0024F5E70120D4
:103D400000F092F804460028F7D1C5F80C0AD8E72D
:103D500000B002500000E0200020704700207047B3
:103D6000014BC3F8040A704700B0025010B5114867
:103D700000F048F800B110BD0F4800F043F80028EB
:103D8000F9D10E4C204600F03DF80028F3D10C4B41
:103D90000C481C6000F036F801460028EBD100F01A
:103DA0002DF8044608B1204610BD00F03FF820462B
:103DB000FAE700BF34010020300100202C01002070
:103DC000240100202801002008B5084800F024F84C
:103DD000074800F021F8074800F01EF8064800F0F8
:103DE0001BF8BDE8084000F00BB800BF340100200C
:103DF000300100202C010020280100200020704705
:103E0000704700BF08B5034B02681B6810689847ED
:103E1000002008BDF400002008B5034B02685B6871
:103E200010689847002008BDF400002070B5094CC8
:103E3000094D2069AB68984718B1084B08485B6882
:103E40009847084AEB68206900211160BDE870407E
:103E5000184700BFE0000020F4000020D800002038
:103E6000A45500008C090020F8B51A4D1A4E0446DE
:103E7000B26828699047E8B9184F3B684CB1A3B1C4
:103E8000012B19D0013B3B602869F368984700205B
:103E9000F8BD43B9124A0121C2F800151149D1F801
:103EA0001029002AFBD101333B60F3682869984749
:103EB0000020F8BD0C48F8BD0A4AD2F81039002B92
:103EC000FBD1074A6FF07E40C2F80035FFF748FF8C
:103ED0003B68D7E7E0000020F40000208C090020B8
:103EE00000A0025000B00250E98FFFFF2DE9F04F13
:103EF0008DB043680293837815469A07804640F157
:103F00000D8100240E78002E00F00A81252E0BD0A2
:103F10004B1C03930134029B4146304698470028CE
:103F2000C0F2F6800399EDE74E788B1C252E0393A3
:103F3000F0D00027B946BB46BBF11F0F38D8A6F119
:103F40002003102B0AD8DFE803F02A0909300909F9
:103F5000092109090928092D09091F00A6F13003C3
:103F6000092B33D92A2E37D11BF0400F55F8043BCB
:103F700040F08280002BA7BF4BF0200B9946C3F185
:103F800000094BF0280B01E04BF0010B039B13F8E9
:103F9000016B0393002ECFD130E04BF0020B4BF0BE
:103FA000040BF3E74BF0080BF0E74BF0100BEDE7D9
:103FB000BBF17F0F19D8A6F13003092BD2D81BF023
:103FC000400F03D00A2101FB0737DFE70A2101FB7D
:103FD00009394BF0200BD9E72E2E06D11BF0400FEC
:103FE00040F09E804BF0400BD0E76C2E31D02BD8A8
:103FF000682E36D06A2E3CD04C2E3AD0002F46F098
:104000002003B8BF2BF04002A3F16501BCBF1FFA2B
:1040100082FB0027022901D9612B2FD1073525F01A
:104020000705DFF8ACA2083507271BF0080F66D09C
:104030000AEB070B56465E4563D1A4EB0A0A06EB72
:104040000A02A9EB07096FE1742E9FD07A2E9DD04A
:10405000D4E71BF0800F18BF4BF4007B4BF0800BB4
:1040600094E71BF4807F18BF4BF4007B4BF4807BFC
:104070008CE74BF4207B89E71F4687E7A6F16301B5
:10408000122900F2F080DFE811F013004F00EE007B
:10409000EE00EE00EE004F00EE00EE00EE00EE004F
:1040A000EE00FE00E900EE00EE001B00EE00AF00A7
:1040B00055F8043B8DF8183001270DF1180AB4E7C4
:1040C00055F804AB834BBAF1000F08BF9A461BF0BA
:1040D000400F14BF39464FF0FF31504600F0E0FF6B
:1040E0000746A2E7029B41462020984700280FDBA5
:1040F000013EB742F6D34C44A41BB14698E74E4666
:10410000F7E716F8010B029B41469847002892DA20
:1041100098F8023043F0040388F802304FF0FF347F
:1041200020460DB0BDE8F08F1BF0800F34D01BF49B
:10413000007F2CD0073525F00705AA4669685AF894
:10414000080B2BF010050029ADB237DA404261EBC5
:10415000410145F480650DF1180B0A235A4600F021
:10416000ABFFA0EB0B0301936B0662D5019B25F01F
:1041700001019F4289B240F3A180002E00F0998096
:1041800015F0100240F09C80BB460D4623E0AA4685
:104190005AF8040BC117D4E7AA461BF4807F5AF8DB
:1041A000041B01D10846F5E71BF4007F15BF48B298
:1041B00008B241F3C01141F3C031C2E750EA010334
:1041C000C9D11BF0400FC6D0002FC4D12BF0110273
:1041D00095B2BB46019740F2064115EA01021CBFA9
:1041E0000BF1010B00222CE02BF010021FFA82FBD6
:1041F0000A231BF0800C49D01BF400711DBF07354A
:1042000025F00705AA46AA461ABF5AF8080B69689E
:104210005AF8040B50EA010545D12BF016051BF0A6
:10422000400FADB242D0002F40D12BF0170295B213
:10423000019715F0100248D0019B002E42D103F1E6
:10424000010B29075AD4EB0706D5D9456FDD019933
:10425000A9EB0B035F18CB465B4649E04BF0100B14
:1042600010237826C5E7782B04D1C6F1780343F0F4
:104270001003BEE7029B4146252098470028FFF621
:1042800047AF023447E608230026B2E7AA461BF4EC
:1042900080715AF8040BBDD01BF400711ABFC0B274
:1042A000614680B2B6E72BF0060295B20DF1180B0D
:1042B00054E725F01105ADB2BB468CE70D46B8E7D3
:1042C0003B460D4603F1020BBBE7DDF804B082E785
:1042D0008C57000085570000CDE904324146029B0F
:1042E000202098470028FFF613AF049B059A01335E
:1042F0009945F1DCA4EB0B01CC189B460AB3029B59
:104300004146302098470028FFF602AF8EB90134AD
:104310002744019B391B994224DC1D465DBB019A51
:10432000A9EB0B09224455461446914435E0019F00
:1043300092E7023441463046029B98470028E7DA6C
:10434000E6E640F206410D42E2D015F0020F14BF3E
:104350002B20202015F4806F04F10104414618BF82
:104360002D20E9E7029B414630209847002804F1C0
:104370000104CEDACCE606AB013D4146585D029B16
:1043800098470028CADAC3E6029B41462020984796
:10439000002804F10104FFF6BBAEA9EB0403002BD7
:1043A000F2DCBFE57047836800EBC101B3F5004F55
:1043B0002CBF51F8220031F81200704700EBC10108
:1043C0008068B0F5004F2CBF41F8223021F8123040
:1043D000704708B50122FFF7E6FFD04008BD8368AB
:1043E000B3F5004F00EBC10108D34B681AB143F09D
:1043F00001034B60704723F00103FAE74B881AB1C1
:1044000043F001034B80704723F00103FAE75300A8
:104410000122FFF7D3BFB0F5004F34BF04230823B8
:10442000481C0833A0EBD300B0FA80F0C0F11F00A5
:1044300070472DE9F0410D4686680446FFF7C9FF35
:10444000B6F5004F014601D3012832D03046FFF7C0
:10445000E2FF04EB80010E6996B9E3680122824015
:104460001343E36002220D612B4629462046FFF7E5
:10447000A5FF032229462046BDE8F041FFF79EBF75
:10448000022231462046FFF78EFF294603460746A3
:104490002046FFF793FF0322334629462046FFF7C5
:1044A0008DFF39462B462046FFF788FF0222314612
:1044B000E1E7BDE8F081B2F5802F2CBF082304238B
:1044C000D21A2DE9F0418C18CD1D25F0070524F0F6
:1044D0000704641B0026E40805602146AC60EE601A
:1044E0002046FFF798FF421D9200013002F10707B6
:1044F0004FEAD707A2F110023146B8BF324605F1A4
:10450000100000F0C5FD3A4631462846FFF77FFF10
:104510003346324631462846FFF750FFA4EB0708E2
:10452000284631460122FFF75AFF42463946FFF737
:104530006EFF3B46324639462846FFF73FFF21468D
:104540002846FFF764FF4346324621462846FFF7D8
:1045500035FF214628460122FFF741FF3946BDE8D5
:10456000F041FFF766BF002070470FB407B504A9FC
:1045700051F8040B0191FBF775FE03B05DF804EBF5
:1045800004B07047038B13F0070305D10368002BB9
:104590000CBF002003207047022B05D1408BB0FADE
:1045A00080F0400980007047012B05D10368002B83
:1045B0000CBF0020052070470020704710B50C4646
:1045C00000B111B96FF0150010BD081D00F093F88F
:1045D0000028F9D1A368032BF6D9F3E72DE9F041C0
:1045E0000D4607461946281D90461E4600F094F8D1
:1045F000044638B13346424629463846A446BDE80B
:10460000F0416047BDE8F08110B4EFF3118220243F
:1046100084F31288BFF36F8F416110BC0121FBF757
:1046200053BE38B50C46054658B151B10B6843B17D
:104630004B6833B11C22002100F02AFD2C610020C0
:1046400038BD6FF01500FBE770B505460E46FFF765
:10465000B5FF041E14DBEFF31182202383F31288CD
:10466000BFF36F8F6B8B2C8B4FF6FF718B4204F077
:10467000070407D182F31188BFF36F8F6FF00A042C
:10468000204670BD022C0CD101336B8382F311885C
:10469000BFF36F8F0023224631462846FFF79EFF67
:1046A000EEE7062C14D8DFE804F004131313041A01
:1046B0000400002333606B683BB9C5E90066ACB900
:1046C00002212846FBF700FEDAE71E606E60F6E77F
:1046D00082F31188BFF36F8F6FF00404D0E782F389
:1046E0001188BFF36F8F6FF08504C9E782F31188DB
:1046F000BFF36F8FC4E7034658B1426802F003026C
:10470000012A03D0032A04D1026812B10020986064
:1047100070476FF0150070474268816002F0030235
:10472000032A4FF0000203460CBF006810465A608F
:1047300070477047FEE7012801D1EFF30583FEF7CC
:10474000D7B901460068FFF7F6BF08B5FBF7CAFF07
:10475000BDE80840FBF7EABF00210120FFF7EBBFEF
:1047600061B662B680F31188BFF36F8F704772B67F
:10477000002383F31188BFF36F8FBFF34F8F30BFD8
:1047800062B6BFF36F8F704772B6002383F3118850
:10479000BFF36F8FBFF34F8F20BF80F31188BFF33C
:1047A0006F8F62B67047202809D9B0F1004F08D842
:1047B0000138B0FA80F0C0F11F00400070470820B7
:1047C00070473E2070470369C9B20C2201FB0233D7
:1047D000186C00F00700704770B5C9B20369EFF3B9
:1047E0001185202484F31288BFF36F8F0C2606FBFB
:1047F0000134246C14F0C00408D0A24206D085F322
:104800001188BFF36F8F4FF0FF3070BD06FB01338F
:1048100001221A6485F31188BFF36F8F436803EB9D
:10482000C1035B6898470020EFE78022FFF7D4BF01
:10483000F8B5069F0469C9B2EFF31186202585F308
:104840001288BFF36F8F0C2505FB0144256C05F022
:10485000070CBCF1010F0CD1276486F31188BFF35C
:104860006F8FC4E90E23436853F831309847002016
:10487000F8BD05F0C005AF4286F31188BFF36F8F16
:104880000CBF6FF077004FF0FF30F1E713B58024D5
:104890000094FFF7CDFF02B010BD10B40069CBB299
:1048A0001C2403FB0400002110BC10470020FDF76E
:1048B000A1BC002000F0CFB91046FEF7F7BB43685B
:1048C0005B68D3F810350B600020704743685B6865
:1048D00002EA010021EA0201C3F80805C3F80C1539
:1048E0000020704743685B680020C3F808157047D4
:1048F00043685B680020C3F80C15704743685A682A
:10490000D2F8043521EA03000B40C2F80805C2F8CA
:104910000C350020704710B503695868F8B188421B
:1049200019D19C6808685860A14200D198600020A5
:1049300008602AB15A680A609A68596002B9996099
:10494000002010E0814206D108682060986881420A
:10495000EDD19C60EBE7044600680028F2D1002A04
:10496000E8D16FF0150010BD30B543681360057ACB
:10497000446804EBC504A34202D36FF0010030BDCC
:104980005C798C4201D00833F0E70020F7E74368F8
:104990001B68D3F88004C3F880047047426813682A
:1049A000D3F8100150B1D269002012780A70C3F810
:1049B0001001D3F8102101221A6070474FF0FF3028
:1049C0007047002A0FDD42681368D3F8100158B110
:1049D0000020C3F81001D269D3F8100112780A70D0
:1049E0000120186070470020704710B543681968AF
:1049F0000369EFF31182202080F31288BFF36F8FD9
:104A00001868002484731B680120D8734FF4800356
:104A1000C1F8043382F31188BFF36F8F10BD0369AF
:104A20001A68012191731B680022DA7370470269CA
:104A300011680346C87B40B15B681B68D3F8580116
:104A400018B100230B6113689889704743681B688D
:104A5000D3F81001003818BF0120704743681B6865
:104A60001022C3F80423704743681B681022C3F860
:104A70000823704743681B684FF40072C3F804238F
:104A8000704743681B684FF40072C3F808237047EF
:104A900038B543681D68D5F804335B02044605D475
:104AA000D5F8040310F0100006D138BDFFF7BFFFA2
:104AB0000028F5D00120F8E72046FFF7C7FF0038AF
:104AC00018BF0120F1E701207047036918680160F1
:104AD0001B685A60704702680346D2F8580140B913
:104AE0005B68DB0706D4D2F82001003818BF01202C
:104AF00070470120704710B4436802691B68D3F8FF
:104B00000413C90517D5D3F82011A1B1EFF3118112
:104B1000202484F31288BFF36F8FD3F8204134B17F
:104B20000024C3F82041D3F820410124DC6081F344
:104B30001188BFF36F8F1468D3F858115CB161B15D
:104B4000002121611468A47B3CB14FF48000C3F8BC
:104B500008031368997310BC7047D3F8241121B16E
:104B60000021C3F82411D3F8243112681368002BF4
:104B7000F1D0516810BC18472DE9F041066933683F
:104B80009C89BFF35B8F94420546A8BF144610333F
:104B9000012753E8002F002A03D143E800700028C2
:104BA000F7D1BFF35B8F0CBF3B4600232BD133689B
:104BB0002246986800F05EFAEFF31188202383F311
:104BC0001288BFF36F8F69680846FFF784FF326869
:104BD00040B91061044688F31188BFF36F8F2046F7
:104BE000BDE8F0810B689268C3F844250022C3F841
:104BF0004845C3F82021D3F82011C3F85821D3F831
:104C000058219F60E7E71C46E9E700F150039B004D
:104C10009BB203F1804303F5883300221A601B68BE
:104C20007047FEF773BF08B5FBF770FCFBF744FD58
:104C3000BDE80840FEF76ABF004700F08EB8C0002C
:104C400000F1804000F5F830C0F81015C0F81425C8
:104C50007047FDF747BFFDF749BAF7B5019001A8C6
:104C6000DDE9084716461D46FDF74CFB019BB6F1F2
:104C7000000C18BF4FF0010C00EB83000B1E18BF97
:104C80000123002D43EA4C0314BF4FF00C0C4FF0EE
:104C9000000C002C43EA0C0314BF4FF4E06C4FF0FF
:104CA000000C002F43EA0C03D0F8002714BF4FF488
:104CB000403C4FF0000C43EA0C0322EA030301B12D
:104CC00009780EB13678760019430DB12D78AD0014
:104CD00031430CB12478240229430FB13F783F04BB
:104CE0000C433C43C0F8004703B0F0BD1FB50DF1C5
:104CF0000F03019300238DF80F1000931A461946F5
:104D0000FFF7ABFF05B05DF804FB38B50546084674
:104D10000C46FDF749FBB0B10846FDF739FB90B9E9
:104D20000846FDF729FB2A6801238340C2F80833AF
:104D30002A6803B202EB8303D3F8102522F00302A2
:104D4000C3F8102538BD20460021BDE83840FFF7E4
:104D5000CDBFFDF7AFBBFFF7D8BF08B1FCF790B9E7
:104D60007047704740B1C368587810F001001EBF0B
:104D70001878B0FA80F040097047EFF311832023D0
:104D800083F31288BFF36F8FFEE708B5FFF7F5FFD7
:104D900010B5D0E9003433B90020E268537843F00D
:104DA0000103537010BD204698470028F4D0002816
:104DB000B8BF4042E368FF28A8BFFF201870ECE7A7
:104DC00000F066B900F056B970474169836843EA5C
:104DD000010212F003020FD1C2600269013A01FB25
:104DE000023382689A4201D900207047C2681A6073
:104DF0004269C3609B1AF4E76FF01500704710B565
:104E0000C0E904320023816083610446FFF7DDFFBF
:104E10000028A8BFC4E9004410BDF8B504460D46FB
:104E2000EFF31186202383F31288BFF36F8FC768D7
:104E30006FB900F0C1F850B18767456100F06EF8B6
:104E4000314604F10800BDE8F840FEF747BBE368CF
:104E50002B60A369E560013BA36186F31188BFF372
:104E60006F8FF8BD08B52024EFF3118384F3128807
:104E7000BFF36F8FFFF77BFCF6E790F90E308B42A4
:104E800001D0FEF7E7BA0020704703460020C3E9CF
:104E90000200C3E900337047EFF30580003818BF04
:104EA00001207047FEF72CBBD0E9003213605A6036
:104EB0000023C0E90033704708B5FFF7F5FF437BD7
:104EC00023F0020343730023836008BD38B5044612
:104ED0000D46FEF79FF9637B43F002036373E5B170
:104EE000A5602B689D4209D16B68C4E900531C6022
:104EF0006C6012E06A689A42F6D01B68002BF3D00F
:104F000094F90E2093F90E108A42F3D09142F1DD0C
:104F10005A68C4E9003214605C6038BD10B5EFF324
:104F20001184202383F31288BFF36F8FFEF78AF971
:104F300084F31188BFF36F8F10BD10B5044618308D
:104F400000F077F8EFF31181202383F31288BFF389
:104F50006F8F627B12F0100204D081F31188BFF3CF
:104F60006F8F10BD2046BDE81040FEF79FB938B5E1
:104F70000446EFF31185202383F31288BFF36F8F6C
:104F8000437B13F0280F0BD183680BB1FFF794FF1D
:104F9000637B51B903F0FB0363732046FEF752F9BC
:104FA00085F31188BFF36F8F38BD03F0EB03F3E790
:104FB00001211838FFF7DBBF38B5EFF31185202347
:104FC00083F31288BFF36F8F0468A0420DD034B111
:104FD0002046FFF771FF04F1180000F02AF885F36E
:104FE0001188BFF36F8F204638BD0024F7E7EFF339
:104FF0001181202282F31288BFF36F8F027BD207C8
:105000000CD581F31188BFF36F8F002383F31188D0
:10501000BFF36F8F0423184602DF7047437B1B07E3
:1050200004D581F31188BFF36F8F70470122FEF71B
:105030003DB910B5EFF31184202282F31288BFF33B
:105040006F8F03683BB1FEF719FC002084F31188D1
:10505000BFF36F8F10BD6FF01500F7E708B5FEF7CF
:105060002BFD08BD10B400F10C04C0E9034410BCD2
:10507000FFF721BA0A44914200F1FF3300D1704793
:1050800010B511F8014B03F8014F9142F9D110BD51
:1050900002440346934200D1704703F8011BF9E72D
:1050A00010B5024601448A42134603D01C780132EF
:1050B000002CF8D1181A10BDF0B5C3F1370704461B
:1050C000FFB203F01F031046082BE6B233D0102BBB
:1050D0003ED06508A40844EA817445EAC1752D19DB
:1050E0004FEA910242EB5102290941EA02716D181F
:1050F00042EB1212290A41EA02616D1842EB1222B8
:10510000290C41EA02416D1842EB1242AD1842F1FE
:105110000002EC0844EA4274D10804EB8402A6EBD6
:105120004205EDB2092D0CD90134A5F10A0541F172
:105130000001EDB212E0E40844EA417406F007050C
:10514000C908303554EA010200F8015BBCD1F0BD5A
:10515000240944EA017406F00F050909092D84BFEA
:10516000ED19EDB2EDE7000001480068704700005E
:10517000980800208CAFFF7F010000003D10000068
:1051800000000000B9110000DC510000752D000086
:1051900000000000E93A00000000000021150000B6
:1051A000F05100002115000004520000951000008D
:1051B00000000000234C000000000000FD1800006B
:1051C00018520000651C00000000000019100000CB
:1051D00000000000274C00000000000021570000E4
:1051E0001C5400002C54000038010020C808002086
:1051F0003057000048540000785400003A01002065
:105200001C0900203E570000605400007854000044
:105210003C01002028090020545700009C54000045
:10522000E05400003E010020240000209D220000E8
:10523000394C0000000000005947000018520000DF
:10524000F74A00000000000059470000000000007D
:1052500059470000000000005947000029290000BC
:10526000394C000000000000594700000000000019
:1052700059470000000000005947000000000000EE
:1052800059470000000000005947000000000000DE
:1052900059470000000000005947000000000000CE
:1052A00059470000000000005947000000000000BE
:1052B0005947000000000000F51C0000000000003D
:1052C000594700000000000059470000000000009E
:1052D000594700000000000059470000000000008E
:1052E000594700000000000059470000000000007E
:1052F000594700000000000059470000000000006E
:10530000594700000000000059470000000000005D
:10531000594700000000000059470000000000004D
:10532000594700000000000059470000000000003D
:10533000594700000000000059470000000000002D
:10534000594700000000000059470000000000001D
:10535000594700000000000059470000000000000D
:1053600059470000000000005947000000000000FD
:1053700059470000000000005947000000000000ED
:1053800059470000000000005947000000000000DD
:1053900059470000000000005947000000000000CD
:0C53A000594700000000000059470000C1
:1053B0000338FDD8704700000000000035470000AA
:1053C0001C000020140000200C0000200000000041
:1053D0000400002025060000190500006D050000EE
:1053E000CD050000000000200000000000000B06BA
:1053F00002000000F8530000000000000C570000FD
:1054000026000207000000201457000022000B11A4
:105410004111000011110000000000009112000075
:1054200085110000AD480000B348000011120000D3
:105430002B4800008D48000000000000C747000016
:105440000000000000000000FFFF0000000300500B
:1054500000000000010000000060004000000000AB
:10546000FFFFFFFF000000500000000000000000F0
:105470000060004000000000B5150000BF480000BB
:10548000CD480000E5480000F1480000FD4800005C
:105490002114000017490000000000000020004017
:1054A0000100000000000000BC54000000000010DB
:1054B00001000000720B0020710B00200020004052
:1054C000C854000001000000D05400000400000097
:1054D0000D000000110000020F0600011406000379
:1054E0009D490000491800008F490000794B0000D9
:1054F000C3490000EB4900001F4A00002F4A00008A
:105500005D4A0000694A00002F4A00004D4A000031
:10551000754A0000834A0000914A0000C74A000013
:10552000CB4A00007C5100007C510000C4510000B7
:10553000CC510000DC510000DC510000FF8FFFFF68
:10554000FF8FFFFFFE8FFFFFFE8FFFFFFD8FFFFF2F
:10555000FC8FFFFFFC8FFFFF6D757465785F6672CF
:1055600065652063616C6C65642077697468204EA2
:10557000554C4C20706172616D657465720000005D
:1055800043616E277420696E697469616C697A651C
:10559000206D757465782C20776173204E554C4CC6
:1055A0000D0A0000436F756C64206E6F74206C6F81
:1055B000636B20706F7765722073617665206D75FF
:1055C000746578005541525420646576696365209E
:1055D0006E6F7420666F756E6421005541525420C1
:1055E00064657669636520646F6573206E6F7420EF
:1055F000737570706F727420696E746572727570F5
:10560000742D64726976656E204150490A004865C0
:105610006C6C6F212049276D20796F75722065634E
:10562000686F20626F742E0D0A0054656C6C206DDB
:105630006520736F6D657468696E6720616E6420A4
:10564000707265737320656E7465723A0D0A004559
:1056500063686F3A20002A2A2A20426F6F74696EAD
:1056600067206E524620436F6E6E6563742053440C
:105670004B2076322E392E302D373738376232367E
:105680003439383430202A2A2A0A002A2A2A205576
:1056900073696E67205A6570687972204F5320765F
:1056A000332E372E39392D316638663364633239FB
:1056B000313432202A2A2A0A006D757465785F69B0
:1056C0006E69742063616C6C65642077697468200E
:1056D0004E554C4C20706172616D6574657200436B
:1056E0006F756C64206E6F7420616C6C6F63617495
:1056F00065206D75746578206265666F72652069D6
:105700006E697469616C697A696E6700464C4153D1
:10571000485F30005352414D5F30000000010000EF
:1057200000636C6F636B40343030303030303000A9
:105730006770696F4035303030303330300067701B
:10574000696F4035303030303030300000010203B6
:1057500004050607756172744034303030323030E1
:1057600030000000000000010100000000000020E7
:105770003030303030303030303030303030000188
:105780006D61696E00286E756C6C29002A666C6FFD
:1057900061742A0067450000540100203A000000AF
:1057A000680100203A000000400100203A0000009B
:1057B0007C0100203A0000003400002000000000BE
:1057C00000000000000000000000000000000000D9
:1057D000730B00202000000000000000000000000B
:1057E00000000000000000000000000000000000B9
:1057F00000000000000000000000000000000000A9
:105800000000000000000000000000000000000098
:105810000000000000000000000000000000000088
:105820000000000000000000000000000000000078
:105830000000000000000000000000000000000068
:105840000000000000000000000000000800000050
:10585000FF00000000000000030000000000000046
:10586000FFFF0F00D0000020D0000020000000004B
:10587000453B00001C010020140100200C01002009
:105880000000000004010020613C0000AD3B00006E
:10589000E13B0000293C00007C0900203A00003A6E
:1058A000800900203A00003A840900203A00003ABA
:1058B000880900203A00003A2C010020F000002066
:1058C000E8000020E4000020E000002000000000CC
:1058D0000000000040010020400100200000000006
:1058E000000000000E0000005401002054010020C0
:1058F00000000000000000000E0000006801002011
:105900006801002000000000000000000E00000000
:105910007C0100207C01002000000000000000004D
:105920000E000000900100209001002020000000E7
:105930000A000000C0190020001B0020C019002030
:10594000C0190020000000000000000015E015E074
:00000001FF
